:0200000480007A
:100000006F00C004732F2034930F8000630AFF0336
:10001000930F90006306FF03930FB0006302FF038A
:10002000170F0080130F0FFE63040F0067000F000F
:10003000732F203463540F006F00400093E19153FD
:10004000171F000023203FFC6FF09FFF732540F136
:1000500063100500970200009382020173905230F2
:10006000735000189702000093820202739052307E
:10007000B70200809382F2FF7390023B9302F0017B
:100080007390023A9702000093828201739052307B
:100090007350203073503030735040309301000063
:1000A00097020000938242F67390523013051000BD
:1000B0001315F501634C05000F00F00F93011000BC
:1000C0009308D0051305000073000000970200801C
:1000D000938242F3638E020073905210B7B2000015
:1000E000938292107390223073232030E39862F44D
:1000F00073500030970200009382420173901234D3
:10010000732540F1730020309300000013010000BC
:1001100033872040930E0000930120006316D74BD5
:10012000930010001301100033872040930E00004D
:1001300093013000631AD749930030001301700017
:1001400033872040930EC0FF93014000631ED747C2
:10015000930000003781FFFF33872040B78E0000F7
:10016000930150006312D747B700008013010000CD
:1001700033872040B70E0080930160006316D74597
:10018000B70000803781FFFF33872040B78E0080A3
:1001900093017000631AD743930000003781000079
:1001A0001301F1FF33872040B78EFFFF938E1E00AF
:1001B00093018000631AD741B70000809380F0FF5D
:1001C0001301000033872040B70E0080938EFEFF9E
:1001D00093019000631AD73FB70000809380F0FF2F
:1001E000378100001301F1FF33872040B78EFF7F76
:1001F0009301A000631AD73DB7000080378100004B
:100200001301F1FF33872040B78EFF7F938E1E00CE
:100210009301B000631AD73BB70000809380F0FFD2
:100220003781FFFF33872040B78E0080938EFEFF1B
:100230009301C000631AD739930000001301F0FF47
:1002400033872040930E10009301D000631ED737F0
:100250009300F0FF1301100033872040930EE0FF5E
:100260009301E0006312D7379300F0FF1301F0FF12
:1002700033872040930E00009301F0006316D735BA
:100280009300D0001301B000B3802040930E2000F3
:1002900093010001639AD0339300E0001301B00092
:1002A00033812040930E300093011001631ED13141
:1002B0009300D000B3801040930E00009301200102
:1002C0006394D031130200009300D0001301B000FA
:1002D000338720401303070013021200930220000B
:1002E000E31452FE930E200093013001631ED32DC0
:1002F000130200009300E0001301B0003387204098
:1003000013000000130307001302120093022000E1
:10031000E31252FE930E3000930140016316D32B7B
:10032000130200009300F0001301B0003387204057
:100330001300000013000000130307001302120053
:1003400093022000E31052FE930E400093015001EF
:10035000631CD327130200009300D0001301B000E8
:10036000338720401302120093022000E31652FE4E
:10037000930E2000930160016318D725130200003B
:100380009300E0001301B000130000003387204009
:100390001302120093022000E31452FE930E300069
:1003A000930170016312D723130200009300F00041
:1003B0001301B00013000000130000003387204039
:1003C0001302120093022000E31252FE930E40002B
:1003D00093018001631AD71F130200009300D0001D
:1003E000130000001301B0003387204013021200F5
:1003F00093022000E31452FE930E2000930190011B
:100400006314D71D130200009300E00013000000E6
:100410001301B000130000003387204013021200C4
:1004200093022000E31252FE930E30009301A001CC
:10043000631CD719130200009300F00013000000A2
:10044000130000001301B000338720401302120094
:1004500093022000E31252FE930E40009301B0017C
:100460006314D717130200001301B0009300D000EB
:10047000338720401302120093022000E31652FE3D
:10048000930E20009301C0016310D71513020000E2
:100490001301B0009300E0001300000033872040F8
:1004A0001302120093022000E31452FE930E300058
:1004B0009301D001631AD711130200001301B00099
:1004C0009300F00013000000130000003387204069
:1004D0001302120093022000E31252FE930E40001A
:1004E0009301E0016312D70F130200001301B00063
:1004F000130000009300D000338720401302120045
:1005000093022000E31452FE930E20009301F001A9
:10051000631CD70B130200001301B000130000008E
:100520009300E00013000000338720401302120004
:1005300093022000E31252FE930E3000930100025A
:100540006314D709130200001301B0001300000068
:10055000130000009300F0003387204013021200C4
:1005600093022000E31252FE930E4000930110020A
:10057000631CD705930010FF33011040930EF00069
:10058000930120026312D1059300000233810040E1
:10059000930E0002930130026318D103B3000040B0
:1005A000930E0000930140026390D003930000017A
:1005B0001301E00133802040930E000093015002AC
:1005C0006314D001631030020F00F00F638001004C
:1005D0009391110093E111009308D0051385010058
:1005E000730000000F00F00F930110009308D00576
:1005F0001305000073000000731000C0000000002D
:0406000000000000F6
:1010000000000000000000000000000000000000E0
:1010100000000000000000000000000000000000D0
:1010200000000000000000000000000000000000C0
:1010300000000000000000000000000000000000B0
:081040000000000000000000A8
:040000058000000077
:00000001FF
